:10000000000008308A00ED2DFF00030E8301A100DF
:100010000A08A0008A010408A2007708A300780853
:10002000A4007908A5007A08A6007B08A70083131E
:1000300083128B1D1D280B183C288C308400001C5B
:1000400023280C183F288C308400801C29288C1809
:100050004228220884002308F7002408F800250815
:10006000F9002608FA002708FB0020088A00210E64
:100070008300FF0E7F0E09008A110A12CB288A1115
:100080000A12BA298A110A12222A0A108A100A119F
:100090008207003400340134003402340034063462
:1000A00000340A3400340F340034163400341E3463
:1000B000003427340034313400343C3400344934C3
:1000C00000345634003465340034743400348534DC
:1000D000003496340034A8340034BB340034CF34B8
:1000E0000034E4340034F93400340F34013425345E
:1000F00001343C340134543401346B3401348434DD
:1001000001349C340134B5340134CE340134E73445
:1001100001340034023419340234323402344B34A2
:100120000234643402347C34023495340234AC3406
:100130000234C4340234DB340234F1340234073480
:1001400003341C3403343134033445340334583419
:1001500003346A3403347B3403348C3403349B34E7
:100160000334AA340334B7340334C4340334CF34EF
:100170000334D9340334E2340334EA340334F1343D
:100180000334F6340334FA340334FE340334FF34D6
:10019000033400340434060830390317A900290851
:1001A000031342020319B129031729080313C200DC
:1001B000031729080339AA00031389000608430618
:1001C0001039031D4929F701061AF71606087706A4
:1001D0002039031D1629C408031D0D29C508031D58
:1001E0000D29C608031D0D29C708031D0D2901305F
:1001F0004C02C4004D08C5000030031C0130C5028C
:100200004E08C6000030031C0130C6024F08C7006C
:100210000030031C0130C7021529FF30C407031C3E
:10022000C507031CC607031CC707482901304C0239
:10023000F7004D08F8000030031C0130F8024E08AA
:10024000F9000030031C0130F9024F08FA000030B9
:10025000031C0130FA0277084402031D4029780884
:100260004502031D402979084602031D40297A08EA
:100270004702031D4029C701C601C501C401482921
:100280000130C4070318C50A0319C60A0319C70AAF
:10029000B1294312061A4316F701061AF716060883
:1002A00077062039031D872901304C02F7004D08DD
:1002B000F8000030031C0130F8024E08F90000304D
:1002C000031C0130F9024F08FA000030031C013012
:1002D000FA0277084402031D7E2978084502031DAF
:1002E0007E2979084602031D7E297A084702031DEC
:1002F0007E29C701C601C501C40186290130C40792
:100300000318C50A0319C60A0319C70AB129C40884
:10031000031DA929C508031DA929C608031DA9296C
:10032000C708031DA92901304C02C4004D08C500AF
:100330000030031C0130C5024E08C6000030031C0B
:100340000130C6024F08C7000030031C0130C7024D
:10035000B129FF30C407031CC507031CC607031CD3
:10036000C707881CB5298810B62988140B108A1174
:100370000A122928FC08031DC029FD080319C529F4
:100380007C080319FD03FC031E2A71088316AA07C3
:1003900072080318720FAB0773080318730FAC07CA
:1003A00074080318740FAD0783120317A901AA017B
:1003B000831603132C0883120317AB008316031351
:1003C0002D0883120317AC00A908031DF029AA0801
:1003D000031DF029AB08031DF029AC080319142AEA
:1003E000FF3083160313AA020318AB020030031C6C
:1003F0000130AC020030031C0130AD020130831229
:100400006E020317A90003136F080317AA00003038
:10041000031C0130AA022A0803138F0003172908BE
:1004200003138E00192A031703136F088F006E0839
:100430008E007608FD007508FC0029140C108A1146
:100440000A1229288316A408031D292AA5080319BE
:100450002E2A24080319A503A4035B2A2808831263
:10046000910083162708A5002608A4008312081C03
:100470003B2A08103C2A081454084402D8004508B6
:10048000D9005508031C550FD9024608DA00560852
:10049000031C560FDA024708DB005708031C570FEE
:1004A000DB024708D7004608D6004508D5004408B7
:1004B000D400A914831683128C108A110A122928D9
:1004C0008316690803194B2B831203179800100831
:1004D000031D6D2A831603134B2B9802031C782AE5
:1004E0007F309807031C772A831603134B2B842A2B
:1004F0008130980203187F2A831603134B2B031DA8
:10050000842A831603134B2B1808F700F801F9010E
:10051000FA019701831603136A08831203179600E2
:100520009617831603136B0883120317950083161F
:1005300003136C08831203179400193098001308F2
:1005400094020318B32A013095020318B32A9602C5
:100550000318B32A97020318B32A970A960A950A32
:1005600013089407E52A120895020318CE2A0130D1
:1005700096020318CE2A97020318CE2A970A960AE3
:100580001208950713089407031CE52A950A031D12
:10059000E52A960A031DE52A970AE52A11088038FC
:1005A00096020318E42A013097020318E42A970AF6
:1005B00011088038960712089507031CC22A960A6C
:1005C000031DC22A970AC22A7A14980BE82AF32A32
:1005D0000310940D950D960D970D0310FA0DF90D5E
:1005E000F80D990D9F2A191CFB2A0310F80CF90C21
:1005F000FA0C990C002BF70B002B831603134B2BD3
:10060000991B292B0310940D950D960D970D13082A
:1006100094020318152B013095020318152B96022E
:100620000318152B9702031C3B2B12089502031885
:10063000202B013096020318202B9702031C3B2B22
:100640001108803896020318292B01309702031CE9
:100650003B2BFA0A031D3B2BF90A031D3B2BF80A1F
:10066000031D3B2BF70A031D382B831603134B2B5B
:10067000F80CF90CFA0C831603136A08831203179B
:10068000980011089806981F472BF817512BF8135C
:10069000512B83160313F701F801F901FA018312B4
:1006A00003170313003483166A08ED00831203173F
:1006B000110883160313ED06ED1F632B03110310BE
:1006C000EA1B0314A62B6A08ED0083120317100817
:1006D00083160313EE006908EE020319752BED1F54
:1006E000A62B0308013A8300A62B831203171108D7
:1006F00083160313EE006A08EE020319852BED1F23
:10070000A62B0308013A8300A62B831203171208B5
:1007100083160313EE006B08EE020319952BED1FF1
:10072000A62B0308013A8300A62B83120317130894
:1007300083160313EE006C08EE020319A52BED1FC0
:10074000A62B0308013A8300A62B03108312003462
:100750008E30F70083166908F7026A08F9006B0803
:10076000F800F917F7080319C02B0310F908031D47
:10077000BC2BF8080319C02BF90CF80CF70BB52BA0
:10078000EA1FC72BF809F909F80A0319F90A8312B5
:1007900000348E30F70083166E08F8006D08F900FB
:1007A000FA01F808031DDE2B7908F800F90108307A
:1007B000F702F808031DDE2BF701E62B0310F81BE8
:1007C000E52BF90DF80DF703DE2BF8138312003437
:1007D0008030831CEE2B03179506031303179A0131
:1007E0009B01110899001508990610080319DC2CC3
:1007F0009800F70014080319E52C98020319812CBE
:10080000031C3F2C15089E009E1716089D00170814
:100810009C009B0103109E0C9D0C9C0C9B0C980B48
:10082000092C991F162C1A14F92C1A1018101A16C4
:100830001330840083170E2D1A12991B292C181CB3
:10084000342C9E0C9D0C9C0C9B0CF70A0319F42C69
:10085000342C9E1B372C03109B0D9C0D9D0D9E0D63
:10086000F7030319F42C292C1A17A12C1A131108B9
:100870009900991F3D2C9E17ED2C9E13ED2C14080A
:100880009800F7001008980211089E009E171208A1
:100890009D0013089C009B0103109E0C9D0C9C0C5A
:1008A0009B0C980B4B2C991F582C9A14F92C9A10CE
:1008B00018109A161730840083170E2D9A12991B60
:1008C0006B2C181C762C9E0C9D0C9C0C9B0CF70A18
:1008D0000319F42C762C9E1B792C03109B0D9C0D78
:1008E0009D0D9E0DF7030319F42C6B2C9A17A12C68
:1008F0009A1315089900991F7F2C9E17ED2C9E13B3
:10090000ED2C15089E009E1716089D0017089C00E8
:10091000991F8E2C9E131A15F92C1A119B01181071
:100920001330840083170E2D991BB72C11089900E2
:10093000181CA12C9E0C9D0C9C0C9B0CF70A0319F7
:10094000F42C9B1FB22C9C0A031DB22C9D0A031D84
:10095000B22C9E0A031DB22C9E0C9D0C9C0CF70A17
:100960000319F42C1A1B362C9A1B782CD62C8030A9
:100970009E069E1FBF2CF92C15089900CC2C11083F
:1009800099009E08031DCC2C9D08031DCC2C9C08AF
:10099000031DCC2CF701ED2C9E1BD62C03109B0DB8
:1009A0009C0D9D0D9E0DF70BCC2CF42C991FDA2C71
:1009B0009E17ED2C9E13ED2C1408F70015089E00D1
:1009C00016089D0017089C00ED2C1008F700110870
:1009D0009E0012089D0013089C001E08F8001D08C8
:1009E000F9001C08FA002C2DF701F801F901FA01B1
:1009F0002C2D9B019C099D099E099B099B0A031DA7
:100A0000072D9C0A031D072D9D0A03199E0A1A181B
:100A1000152C9A18572C1A198D2CBC2C00089C07E1
:100A2000031C182D9D0A031D182D9E0A0319181466
:100A3000840300089D07031C202D9E0A0319181427
:100A400084030008801F803A9E07031818141A1A9E
:100A50001C2C9A1A5E2C942C0313003403171008D4
:100A600003199F2D9800140803199F2D9807031848
:100A7000402D7F309802031C9F2D03199F2D442D7C
:100A80008130980703189F2D1808F700F801F90125
:100A9000FA0111089C009C1712089B0013089A0089
:100AA0001830980099011A1C6D2D1708FA07031CBD
:100AB0005F2DF90A031D5F2DF80A0319991716080F
:100AC000F907031C662DF80A0319991715089200F7
:100AD00092171208F80703189917990DF80CF90CDA
:100AE000FA0C9C0C9B0C9A0C0310980B522D0130A5
:100AF000F70703189F2DF81B842D9C0DFA0DF90D97
:100B0000F80DF70303199F2D9C1F952DFA0A031D5D
:100B1000952DF90A031D952DF80A031D952DF80C46
:100B2000F90CFA0CF70A03199F2D11089900150802
:100B30009906991F9D2DF817A32DF813A32DF701E2
:100B4000F801F901FA0103130034831668105C08F8
:100B5000E1005B08E0005A08DF005908DE005C088D
:100B6000EC005B08EB005A08EA005908E900831220
:100B70000317930192019101900103135323031C66
:100B8000C72D831668145F08803ADF00831283162E
:100B90006108EC006008EB005F08EA005E08E9000D
:100BA000831203179301920191018E309000031379
:100BB00053230318DD2D031DFA2D83166108EC0065
:100BC0006008EB005F08EA005E08E9008312A823D2
:100BD00079088316EE007808ED008312C9237A089D
:100BE0008316E5007908E4007808E3007708E2005E
:100BF000F42E831283166108EC006008EB005F0896
:100C0000EA005E08E90080308312031793009630F3
:100C10009200183091009630900003135323031C68
:100C2000EB2E83166108EC006008EB005F08EA0019
:100C30005E08E900831203179301920191018E303F
:100C40009000031360227A088316EC007908EB0009
:100C50007808EA007708E9008312A8237908831648
:100C6000E7007808E6006108EC006008EB005F0828
:100C7000EA005E08E90083120317930192019101D3
:100C80008E3090000313602277088316E9007808FD
:100C9000EA007908EB007A08EC006708EE006608C5
:100CA000ED008312C923831483166C088312031783
:100CB0009300831603136B088312031792008316A5
:100CC00003136A088312031791008316031369083C
:100CD0008312031790007A08970079089600780825
:100CE0009500770894000313E823031793019201FA
:100CF00091018E3090007A08970079089600780864
:100D000095007708940003132E257A088316E100D6
:100D10007908E0007808DF007708DE006708EE0059
:100D20006608ED008312C923031793019201910114
:100D30008E3090007A089700790896007808950020
:100D40007708940003132E257A088316E5007908A6
:100D5000E4007808E3007708E2006108EC0060082E
:100D6000EB005F08EA005E08E9008312A823790817
:100D70008316EE007808ED008312C92383108316D2
:100D80006508831203179300831603136408831204
:100D9000031792008316031363088312031791004D
:100DA0008316031362088312031790007A089700D2
:100DB0007908960078089500770894000313E823D3
:100DC0007A088316E5007908E4007808E3007708DC
:100DD000E200F42E831283166108E5006008E40047
:100DE0005F08E3005E08E2006108EC006008EB00C9
:100DF0005F08EA005E08E9008312A82379088316D9
:100E0000EE007808ED008312C9238314831661086D
:100E100083120317930083160313600883120317CA
:100E20009200831603135F08831203179100831641
:100E300003135E088312031790007A08970079085D
:100E4000960078089500770894000313E8237A0841
:100E50008316E1007908E0007808DF007708DE00FB
:100E6000681C352F6308803AE3006108EC006008D5
:100E7000EB005F08EA005E08E900831203179301A4
:100E8000920191019001031353230319A02F83169C
:100E9000681C742FDD08031D742F831465088312EA
:100EA0000317930083160313640883120317920039
:100EB0008316031363088312031791008316031329
:100EC00062088312031790009701960195017F3005
:100ED00094000313E8237A088316E5007908E400F8
:100EE0007808E3007708E20068189F2F5D0B9F2FBA
:100EF0008310650883120317930083160313640895
:100F000083120317920083160313630883120317D7
:100F10009100831603136208831203179000970150
:100F2000960195017F3094000313E8237A08831615
:100F3000E5007908E4007808E3007708E20083120E
:100F400083165C08EC005B08EB005A08EA005908BD
:100F5000E900831203179301920191019001031399
:100F60005323031DB92F8316E501E401E301E201D8
:100F7000831283166208F7006308F8006408F9001A
:100F80006508FA008312003483163E080F39F70013
:100F9000770DC000C00DFC30C005400883128800EA
:100FA00083163E080F39BF00831285000034831674
:100FB0003E0EF700F030F7057708E039C1003E0833
:100FC00001394104BF003E19E92F83120813EB2FAA
:100FD0008316831208178316BE19F22F8312881303
:100FE000F42F83168312881783163E080339C00036
:0E0FF0008312890083163F08831287000034A5
:1010000083164208F9004108F800F90CF80CF90CB5
:10101000F80CF90C780883129500F90C790C30392A
:10102000F7001708CF397704970000348316390882
:101030008312DE00003A03192A28013A03192F28E7
:10104000033A03193428013A03193928073A0319D6
:1010500039283E280330DC000630DD00442801300A
:10106000DC000430DD0044280130DC000530DD0008
:1010700044280A30DC000630DD0044280130DC0062
:101080000530DD004428442883163C088312DF0025
:1010900083163C088312E000E10183163A088312AC
:1010A000E20083163A088312E300E40183163B084A
:1010B000023A831203196F28063A03196F280C3A73
:1010C00003196F28183A03196F28303A03196F284B
:1010D000603A03196F28403A03197B287B280310D4
:1010E00083163B0C8312E7006708E8000130E50037
:1010F0006508E6008028E701E801E501E6018028AF
:101100005F080239023C031DC62861085C078400A1
:1011100083135D1883170008EC00013061075C073A
:10112000840083135D18831700088316BF008312A1
:1011300061085C07840083135D1883170008831619
:101140003F06BD000130831261075C0784008313F2
:101150005D18831700088316BD05831261085C07BC
:10116000840083135D18831700088316BE000130C6
:101170008312610707395C07840083135D188317A6
:10118000000883163E048312EC00FE280130610241
:1011900007395C07840083135D18831700088316E2
:1011A000C000831261085C07840083135D188317F5
:1011B000000883164006BD00831261085C078400A6
:1011C00083135D18831700088316BD058312610819
:1011D0005C07840083135D18831700088316BE0024
:1011E00001308312610207395C07840083135D18A4
:1011F0008317000883163E048312EC006C088316E4
:10120000BE008A118312C4278A1583163D08BE00CA
:101210008A118312D7278A150310640D8316BE0026
:101220003E0A8A11831245208A15FA0083163E0869
:101230008A11831245208A158316BF007A08C000E0
:10124000C2003F08C1008312002000348316B80199
:10125000003085008113F03086000030880018309F
:101260008700013083128800831609108910091144
:10127000831207110C3097007830F800053892007F
:10128000403083169200831295018316BC01013011
:10129000BB008630BA00A030B9009530C400BF3022
:1012A000C3005630C2007430C1003C08D0003B0877
:1012B000CF003A08CE003908CD00B630F700FA0169
:1012C000F901F8014D084E044F045004031D6A292A
:1012D000F70177290310F81B7629CD0DCE0DCF0D20
:1012E000D00DFA0DF90DF80DF70B6A29F8137A08ED
:1012F000EC007908EB007808EA007708E90083122F
:1013000003179301243092007430910092309000C2
:101310008A11031360228A1577088316CD00780896
:10132000CE007908CF007A08D000EC004F08EB001F
:101330004E08EA004D08E9004408831203179300A1
:1013400083160313430883120317920083160313B3
:101350004208831203179100831603134108831276
:10136000031790008A11031360228A157A088316E6
:10137000C0007908BF007808BE007708BD004008AB
:10138000D0003F08CF003E08CE003D08CD00D2017E
:10139000C530D1005208FA005108D3007A08D400B1
:1013A0005008EC004F08EB004E08EA004D08E90039
:1013B0008312031793019201910190018A11031383
:1013C00053238A15031CFC2983165008D8004F08A4
:1013D000D7004E08D6004D08D5005808DC00570845
:1013E000DB005608DA005508D9000130DD008A110B
:1013F0008312A5258A15122A83165008D8004F0893
:10140000D7004E08D6004D08D5005808DC00570814
:10141000DB005608DA005508D900DD018A11831275
:10142000A5258A158316530884008313541883173F
:1014300077088000840A78088000840A7908800090
:10144000840A7A0880005208FA0051088400831345
:10145000521883170008F700840A0008F800840A6D
:101460000008F900840A0008FA00D4010408D30037
:101470005410831B541483145008831203179300D1
:10148000831603134F088312031792008316031366
:101490004E08831203179100831603134D0883121D
:1014A000031790007A08970079089600780895004D
:1014B000770894008A110313E8238A1583165308CA
:1014C00084008313541883177A08CC007908CB0062
:1014D0007808CA007708C9004808EC004708EB0004
:1014E0004608EA004508E9008A118312A8238A15F4
:1014F00079088316A5007808A4002508A700240809
:10150000A6004C08831203179300831603134B089D
:10151000831203179200831603134A0883120317DA
:101520009100831603134908831203179000970153
:10153000960195018F3094008A1103132E258A1588
:101540007A088316CC007908CB007808CA0077089F
:10155000C9004C08EC004B08EB004A08EA004908B7
:10156000E9008A118312A8238A1579088316A90035
:101570007808A800C401C301C201C101043083126C
:10158000ED00F401F301F2015930F100B030EF0049
:10159000B930EE00FD01FC017D30F600F501831647
:1015A000BC010A30BB00FC30BA008030B900C00179
:1015B000BF01BE01BD010130C10040088312CB0054
:1015C00083163F088312CA0083163E088312C9009F
:1015D00083163D088312C800831640088312C70093
:1015E00083163F088312C60083163E088312C50087
:1015F00083163D088312C40083163C088312CF0073
:1016000083163B088312CE0083163A088312CD005E
:10161000831639088312CC00D301D201D10183167D
:1016200041088312D0004708D7004608D600450875
:10163000D5004408D400DB01DA01D901D8016D08D6
:101640008316B9000C108312ED08031D2A2B853078
:101650009000382B6D0B2F2B95309000382B6D0898
:10166000023C031D362BA5309000382BB53090007E
:1016700083160C14B9013030BA00BB018230BC00B3
:10168000831216206F088316BA0083126E08831621
:10169000B9007D08BC007C08BB000C103C08F600BB
:1016A0003B08F5003A088312EF00831639088312CD
:1016B000EE0083160C1483126F088F006E088E00E4
:1016C00083162808831291008B1583160C148C1432
:1016D0000C158C15C03083128B0408148A150A125D
:1016E0005E2E83163A08F801390203187A2B39085E
:1016F000F700862BF7010830BB00B90DF70D3A084B
:1017000077020318F700F80DBB0B7D2B8312003412
:10171000F701F80183163A0803103B18F707F70C96
:10172000F80CBB18F707F70CF80C3B19F707F70C88
:10173000F80CBB19F707F70CF80C3B1AF707F70C76
:10174000F80CBB1AF707F70CF80C3B1BF707F70C64
:10175000F80CBB1BF707F70CF80C83120034DF1FE3
:10176000A42D65086407E400E4080319BB2B67088F
:101770006402031C722DE4080319C22B6808013CA3
:10178000031CAE2CE4016608E5005F080239023C48
:10179000031D3C2CE10A0730E10561085C07840069
:1017A00083135D1883170008EC00013061070739C7
:1017B0005C07840083135D1883170008EC046C0831
:1017C0008316BE008A118312C4278A15013061076F
:1017D00007395C07840083135D1883170008E9004C
:1017E00061085C07840083135D1883170008E9060D
:1017F0000130610707395C07840083135D18831784
:101800000008E90569088316BE008A118312D727EC
:101810008A1540308316B900831267088316BA0010
:101820008312712378088316B9003908BA0083122D
:1018300064088316BB008312882378088316B800D7
:101840000310380DB900390A8A11831245208A1510
:10185000FA00831639088A11831245208A15EA0096
:101860007A08EB006B088316C20083126A0883169D
:10187000C10083120020AD2CE1030730E1056108AF
:101880005C07840083135D1883170008EC000130A7
:10189000610207395C07840083135D188317000811
:1018A000EC046C088316BE008A118312C4278A15C3
:1018B0000130610207395C07840083135D188317C8
:1018C0000008E90061085C07840083135D18831732
:1018D0000008E9060130610207395C0784008313C0
:1018E0005D1883170008E90569088316BE008A1190
:1018F0008312D7278A1540308316B90083126708F0
:101900008316BA008312712378088316B900390848
:10191000BA00831264088316BB00831288237808F8
:101920008316B8000310380DB900390A8A118312E2
:1019300045208A15FA00831639088A11831245203A
:101940008A15EA007A08EB006B088316C20083123E
:101950006A088316C10083120020712DFF308316A0
:10196000BA00831265088316BB00831288237808A7
:10197000E5006708E4005F080239023C031D192DE9
:101980000130610707395C07840083135D188317F2
:1019900000088316BB00831261085C078400831370
:1019A0005D188317000883163B068312E90061085F
:1019B0005C07840083135D1883170008E905690834
:1019C0008316BE008A118312D7278A1540308316EA
:1019D000B900831267088316BA008312712378084E
:1019E0008316B9003908BA00831264088316BB0055
:1019F0008312882378088316B8000310380DB900C5
:101A0000390A8A11831245208A15FA00831639088B
:101A10008A11831245208A15EA007A08EB006B08C8
:101A20008316C20083126A088316C1008312002045
:101A3000712D0130610207395C07840083135D1842
:101A4000831700088316BB00831261085C078400BB
:101A500083135D188317000883163B068312E90081
:101A600061085C07840083135D1883170008E9058B
:101A700069088316BE008A118312D7278A15403061
:101A80008316B900831267088316BA008312712384
:101A900078088316B9003908BA00831264088316DF
:101AA000BB008312882378088316B8000310380D12
:101AB000B900390A8A11831245208A15FA00831663
:101AC00039088A11831245208A15EA007A08EB004A
:101AD0006B088316C20083126A088316C100831242
:101AE0000020A42D40308316B900831267088316A6
:101AF000BA008312712378088316B9008312640830
:101B00008316BA003908BB0083128823780883162D
:101B1000B8000310380DB900390A8A118312452024
:101B20008A15FA00831639088A11831245208A150E
:101B3000EA007A08EB006B088316C20083126A0879
:101B40008316C100831200208A150A12612EF70144
:101B5000F801F901FA018316C401C501C601C701E4
:101B600043084204410440040319E62D2030C80014
:101B70000310BC0DBD0DBE0DBF0DC40DC50DC60DB2
:101B8000C70D43084702031DCF2D42084602031D1F
:101B9000CF2D41084502031DCF2D40084402031CF0
:101BA000E02D4008C4024108031C410FC502420851
:101BB000031C420FC6024308031C430FC702031451
:101BC000F70DF80DF90DFA0DC80BB82DC4308400CF
:101BD000831383128A150A12062F03081F39830004
:101BE0005030F7002030840083138001840AF70B03
:101BF000F52DF101F201F301F401F501F601F8010F
:101C0000F901FA01FB01FC01FD01FE015030F70072
:101C1000A030840083138001840AF70B0B2E603000
:101C2000F7001030840083178001840AF70B142E0C
:101C300083135530F7009030840083178001840AA5
:101C4000F70B1E2E831383160317EE0183138312E3
:101C50000313A001840183131F308305A8152808EE
:101C60008316870083122816280883168700D83029
:101C70009300363083129400831611141F149F149E
:101C80001F159F1107309C00FF308312A800AB0185
:101C9000AC01C101C201C301ED01FE018316AA011D
:101CA000AB01AC01AD01AE01B001B101B201B301B4
:101CB000B401B501B601B70183122629291C6E2F84
:101CC000AF2B5F086039031DBD2E5F0860068039A9
:101CD0008316AF00AF0803198F2E8312E01F7F2EEB
:101CE0008316B901831263088316BA008312680849
:101CF0008316BB008230BC00831216208D2EE51B9C
:101D0000892E650866020318892E0310650CE5000C
:101D10008D2EDF0160088039DF04BC2E831683120C
:101D20005F08600602390319A82EE408031DA72ED8
:101D3000E51BA22E650866020318A22E0310650C8F
:101D4000E500A72E0230DF0660080239DF04BC2E52
:101D5000660865020319BC2EE408031DBC2EE51BB2
:101D6000B92E650866020318B92E0310650CE5004C
:101D7000BC2E0310650DE5006A2F5F086039403CFA
:101D8000031D632F440848028316B80083124908D4
:101D90008316B90083124508031C450FD02ED32E9D
:101DA0008316B90283124A088316BA0083124608C2
:101DB000031C460FDC2EDF2E8316BA0283124B085B
:101DC0008316BB0083124708031C470FE82EEB2E37
:101DD0008316BB02831283163B08BF003A08BE007D
:101DE0003908BD003808BC00831253088316C300AD
:101DF000831252088316C200831251088316C10051
:101E0000831250088316C0008312A72D7A08831608
:101E1000B7007908B6007808B5007708B40035082F
:101E2000AF00B408031D212FB508031D212FB608EC
:101E3000031D212FB708031D212F8312DF01602FFF
:101E40008316B408031D2D2FB508031D2D2FB608CA
:101E5000031D2D2FB7080319612FAF08031D4B2F4A
:101E600083126608E5006808E700DF018316B408FE
:101E7000031D432FB508031D432FB608031D432F31
:101E8000B7080319452F0230462F00308312DF04B4
:101E9000DF17602F83168312E51B522F6608650239
:101EA0000318602F6508F70083162F08F800031940
:101EB0005D2F0310F70DF80B592F77088312E500FB
:101EC00083166B2F83125F086039603C03196A2FF9
:101ED0008A010028831601308312A906A91CA92FA4
:101EE000440848028316B800831249088316B900D3
:101EF00083124508031C450F7E2F812F8316B902DC
:101F000083124A088316BA0083124608031C460F40
:101F10008A2F8D2F8316BA0283124B088316BB00BB
:101F200083124708031C470F962F992F8316BB0275
:101F300083128316B808031DA52FB908031DA52F0A
:101F4000BA08031DA52FBB08031DA62F023083125C
:061F5000A9065E2EAA2F77
:02400E003A373F
:00000001FF
